:020000040000FA
:0A0000000000000025EF00F038D0EA
:0800180085D0096A086EFF0E95
:100020000826092200D0D8A01200030E076EE60EA3
:1000300002D8F5D7076AFE0F066EE86A075AD8A0FD
:1000400012000000060600D0F8D74F0EAF6E240E47
:10005000AC6E900EAB6E00010FEE7FF0ED6AE950D2
:10006000EA10FCE1EF6A0F0EC16E070EB46EC69A7D
:10007000C00E926E936A946E6ED0F2A403D0F29486
:10008000827011009EAA19D0060EAB1412E1E2CFC5
:1000900034F0E1CF33F0352A10EE57F03550E12639
:1000A000000EE222AECFE7FF34C0E2FF33C0E1FF33
:1000B0001100AE50AE50AB98AB8811003550365C95
:1000C00014E0362AEACF07F0E9CF06F000EE57F049
:1000D0003650E926000EEA22EF50066E07C0EAFF0E
:1000E00006C0E9FFD880120004D0E868066ED8A0E8
:1000F00012001200356A366A9D8A9F8AF28EF28C4F
:1001000012009D9A00EE57F0010EF46EF36AF306AA
:10011000000EF45AEE6AF450F310F9E1356A366ACB
:100120009D8A1200F29EE0CF57F2D8CF58F2E8CF66
:1001300059F2F28E0001A192B36AB26AF29E57C2DE
:10014000E0FF58C2D8FF59C2E8FFF28E10009EA807
:10015000FED7AD6E1200040ECA6ECB68BB6A0C0EE1
:10016000BA6E9492040ECA6ECB68BE6A0C0EBD6E57
:100170009494936A94908B800A0E4FDF94908B90A6
:10018000929A898A8A6A94968B86929089809292B2
:10019000898292948984936A8A6A94968B969496BB
:1001A0008B86929089909290898092928992929275
:1001B00089829294899492948984570E2C6E2C5043
:1001C000FF082D6E030ED8A0FF0F2E6E00EE2DF04F
:1001D000CF0EBD16EE38300BBD12ED30F36EEF30A2
:1001E000BE6EF332BE32196A00EE37F0200EEE68B2
:1001F000E82EFDD71A6A2F6A306A316A326A7ADFCE
:1002000080DFCD6AF294F28A870ED56EB16AA19230
:10021000A082B36AB26AD08EA292B10EB16E89EC9E
:1002200008F0252AE86A25B2010F26B0010806E188
:100230002670212A000E2222232224223FDF0A6E6A
:10024000E30E0A5C06E3FE0E0A5C01E20C6A99EF1B
:1002500006F00AAE38D00C6A820E0A5C05E10AC0CC
:100260000CF00D680E682DD0920E0A5C05E10AC0F4
:100270000CF00F68106825D0A20E0A5C05E10AC0D8
:100280000CF0116812681DD0B20E0A5C05E10AC0BC
:100290000CF01368146815D0C20E0A5C04E10AC0A1
:1002A0000CF015680ED0D20E0A5C04E10AC00CF006
:1002B000166807D0E20E0A5C04E10AC00CF0176869
:1002C000186898EF06F00C5204E199EF06F098EFE9
:1002D00006F0820E0C5CD8A479D10D2803E10AC087
:1002E0000DF070D10AC00EF0200E0D5C0DE12F9EB6
:1002F0002FC081FF94968B9694968B861B903A68BC
:100300003968386837685BD1210E0D5C0DE12F9C90
:100310002FC081FF94968B9694968B861B923E6895
:100320003D683C683B684BD1220E0D5C0DE12F9A75
:100330002FC081FF94968B9694968B861B9442686F
:10034000416840683F683BD1230E0D5C0DE12F985A
:100350002FC081FF94968B9694968B861B96466849
:100360004568446843682BD1240E0D5C08E12F9644
:100370002FC081FF94968B9694968B8620D1250E64
:100380000D5C08E12F942FC081FF94968B96949674
:100390008B8615D1260E0D5C08E12F922FC081FFB0
:1003A00094968B9694968B860AD1270E0D5C08E165
:1003B0002F902FC081FF94968B9694968B86FFD0BA
:1003C000280E0D5C08E1309E30C081FF929089902C
:1003D00092908980F4D0290E0D5C08E1309C30C0E9
:1003E00081FF9290899092908980E9D02A0E0D5CCD
:1003F00008E1309A30C081FF929089909290898074
:10040000DED02B0E0D5C08E1309830C081FF929059
:10041000899092908980D3D02C0E0D5C08E13096A3
:1004200030C081FF9290899092908980C8D02D0E23
:100430000D5C08E1309430C081FF929089909290D9
:100440008980BDD02E0E0D5C08E1309230C081FF56
:100450009290899092908980B2D02F0E0D5C08E125
:10046000309030C081FF9290899092908980A7D07F
:10047000300E0D5C08E1319E31C081FF929289926D
:10048000929289829CD0310E0D5C08E1319C31C082
:1004900081FF929289929292898291D0320E0D5C64
:1004A00008E1319A31C081FF9292899292928982B9
:1004B00086D0330E0D5C08E1319831C081FF9292F5
:1004C0008992929289827BD0340E0D5C08E131963C
:1004D00031C081FF929289929292898270D0350EBA
:1004E0000D5C08E1319431C081FF92928992929221
:1004F000898265D0360E0D5C08E1319231C081FFF2
:1005000092928992929289825AD0370E0D5C08E1BC
:10051000319031C081FF92928992929289824FD01C
:10052000380E0D5C08E1329E32C081FF92948994AE
:100530009294898444D0390E0D5C08E1329C32C01B
:1005400081FF929489949294898439D03A0E0D5CFB
:1005500008E1329A32C081FF9294899492948984FE
:100560002ED03B0E0D5C08E1329832C081FF929490
:1005700089949294898423D03C0E0D5C08E13296D4
:1005800032C081FF929489949294898418D03D0E50
:100590000D5C08E1329432C081FF92948994929468
:1005A00089840DD03E0E0D5C08E1329232C081FF8D
:1005B000929489949294898402D099EF06F00D6800
:1005C00098EF06F099EF06F098EF06F0920E0C5CAB
:1005D000D8A45DEF06F00F2804E10AC00FF05BEF2E
:1005E00006F00AC010F01052D8A46ED1200E0F5C95
:1005F0000DE12F9E2FC081FF94968B9694968B864B
:100600001B903A683968386837685BD1210E0F5CF7
:100610000DE12F9C2FC081FF94968B9694968B862C
:100620001B923E683D683C683B684BD1220E0F5CD4
:100630000DE12F9A2FC081FF94968B9694968B860E
:100640001B944268416840683F683BD1230E0F5CB1
:100650000DE12F982FC081FF94968B9694968B86F0
:100660001B9646684568446843682BD1240E0F5C8E
:1006700008E12F962FC081FF94968B9694968B86D7
:1006800020D1250E0F5C08E12F942FC081FF949696
:100690008B9694968B8615D1260E0F5C08E12F92CF
:1006A0002FC081FF94968B9694968B860AD1270E45
:1006B0000F5C08E12F902FC081FF94968B96949643
:1006C0008B86FFD0280E0F5C08E1309E30C081FF82
:1006D0009290899092908980F4D0290E0F5C08E165
:1006E000309C30C081FF9290899092908980E9D0AF
:1006F0002A0E0F5C08E1309A30C081FF92908990F9
:1007000092908980DED02B0E0F5C08E1309830C0CB
:1007100081FF9290899092908980D3D02C0E0F5CAB
:1007200008E1309630C081FF929089909290898044
:10073000C8D02D0E0F5C08E1309430C081FF92903C
:10074000899092908980BDD02E0E0F5C08E1309286
:1007500030C081FF9290899092908980B2D02F0E04
:100760000F5C08E1309030C081FF929089909290A8
:100770008980A7D0300E0F5C08E1319E31C081FF27
:1007800092928992929289829CD0310E0F5C08E1FC
:10079000319C31C081FF929289929292898291D04C
:1007A000320E0F5C08E1319A31C081FF929289923A
:1007B0009292898286D0330E0F5C08E1319831C065
:1007C00081FF92928992929289827BD0340E0F5C43
:1007D00008E1319631C081FF92928992929289828A
:1007E00070D0350E0F5C08E1319431C081FF9292D8
:1007F00089929292898265D0360E0F5C08E131921F
:1008000031C081FF92928992929289825AD0370E9A
:100810000F5C08E1319031C081FF929289929292EF
:1008200089824FD0380E0F5C08E1329E32C081FFC2
:10083000929489949294898444D0390E0F5C08E193
:10084000329C32C081FF929489949294898439D0E9
:100850003A0E0F5C08E1329A32C081FF929489947B
:10086000929489842ED03B0E0F5C08E1329832C0FE
:1008700081FF929489949294898423D03C0E0F5CDA
:1008800008E1329632C081FF9294899492948984CF
:1008900018D03D0E0F5C08E1329432C081FF929473
:1008A0008994929489840DD03E0E0F5C08E13292B7
:1008B00032C081FF929489949294898402D099EFF6
:1008C00006F098EF06F0F7D11AA0F3D1200E0F5CD6
:1008D0002FE12F8E2FC081FF94968B9694968B8656
:1008E0007F0E105C23E21B8010C01DF001EE57F05C
:1008F000D8901D34E926000EEA22EECF04F0EFCFA7
:1009000005F004502124006E05502220016E000ED7
:100910002320026E000E2420036E03C03AF002C0B2
:1009200039F001C038F000C037F001D01B90C1D1C0
:10093000210E0F5C2FE12F8C2FC081FF94968B9698
:1009400094968B867F0E105C23E21B8210C01EF0F3
:1009500001EE57F0D8901E34E926000EEA22EECFC1
:1009600004F0EFCF05F004502124006E0550222042
:10097000016E000E2320026E000E2420036E03C0C1
:100980003EF002C03DF001C03CF000C03BF001D0A1
:100990001B928FD1220E0F5C2FE12F8A2FC081FF77
:1009A00094968B9694968B867F0E105C23E21B8424
:1009B00010C01FF001EE57F0D8901F34E926000E4A
:1009C000EA22EECF04F0EFCF05F004502124006EB0
:1009D00005502220016E000E2320026E000E2420FE
:1009E000036E03C042F002C041F001C040F000C0FD
:1009F0003FF001D01B945DD1230E0F5C2FE12F88B7
:100A00002FC081FF94968B9694968B867F0E105CF8
:100A100023E21B8610C020F001EE57F0D89020345E
:100A2000E926000EEA22EECF04F0EFCF05F00450E5
:100A30002124006E05502220016E000E2320026E3C
:100A4000000E2420036E03C046F002C045F001C032
:100A500044F000C043F001D01B962BD1240E0F5C54
:100A600008E12F862FC081FF94968B9694968B86F3
:100A700020D1250E0F5C08E12F842FC081FF9496B2
:100A80008B9694968B8615D1260E0F5C08E12F82EB
:100A90002FC081FF94968B9694968B860AD1270E51
:100AA0000F5C08E12F802FC081FF94968B9694965F
:100AB0008B86FFD0280E0F5C08E1308E30C081FF9E
:100AC0009290899092908980F4D0290E0F5C08E171
:100AD000308C30C081FF9290899092908980E9D0CB
:100AE0002A0E0F5C08E1308A30C081FF9290899015
:100AF00092908980DED02B0E0F5C08E1308830C0E8
:100B000081FF9290899092908980D3D02C0E0F5CB7
:100B100008E1308630C081FF929089909290898060
:100B2000C8D02D0E0F5C08E1308430C081FF929058
:100B3000899092908980BDD02E0E0F5C08E13082A2
:100B400030C081FF9290899092908980B2D02F0E10
:100B50000F5C08E1308030C081FF929089909290C4
:100B60008980A7D0300E0F5C08E1318E31C081FF43
:100B700092928992929289829CD0310E0F5C08E108
:100B8000318C31C081FF929289929292898291D068
:100B9000320E0F5C08E1318A31C081FF9292899256
:100BA0009292898286D0330E0F5C08E1318831C081
:100BB00081FF92928992929289827BD0340E0F5C4F
:100BC00008E1318631C081FF9292899292928982A6
:100BD00070D0350E0F5C08E1318431C081FF9292F4
:100BE00089929292898265D0360E0F5C08E131823B
:100BF00031C081FF92928992929289825AD0370EA7
:100C00000F5C08E1318031C081FF9292899292920B
:100C100089824FD0380E0F5C08E1328E32C081FFDE
:100C2000929489949294898444D0390E0F5C08E19F
:100C3000328C32C081FF929489949294898439D005
:100C40003A0E0F5C08E1328A32C081FF9294899497
:100C5000929489842ED03B0E0F5C08E1328832C01A
:100C600081FF929489949294898423D03C0E0F5CE6
:100C700008E1328632C081FF9294899492948984EB
:100C800018D03D0E0F5C08E1328432C081FF92948F
:100C90008994929489840DD03E0E0F5C08E13282D3
:100CA00032C081FF929489949294898402D00F6813
:100CB00040D00F683DD03DD03BD0A20E0C5C0BE184
:100CC000112803E10AC011F004D00AC012F06FD954
:100CD0002FD02FD02DD0B20E0C5C0AE1132803E1E7
:100CE0000AC013F003D00AC014F080D922D020D05B
:100CF000C20E0C5C07E1152803E10AC015F070D99B
:100D000018D016D0D20E0C5C07E1162803E10AC0F9
:100D100016F06AD90ED00CD0E20E0C5C09E117284F
:100D200003E10AC017F003D00AC018F05BD901D064
:100D300004D9040E2B5CD8B0F8D02750215C285081
:100D40002258295023582A502458D8A0E0D02A8E5F
:100D50002B5235E11BB00CD02F9E2FC081FF9496F3
:100D60008B9694968B863A6839683868376826D0AF
:100D70002F7E2FC081FF94968B9694968B8601EEE2
:100D800057F0D8901D34E926000EEA22EECF04F089
:100D9000EFCF05F004502124006E05502220016E93
:100DA000000E2320026E000E2420036E03C03AF0D2
:100DB00002C039F001C038F000C037F0A7D0010EF2
:100DC0002B5C35E11BB20CD02F9C2FC081FF949679
:100DD0008B9694968B863E683D683C683B6826D02F
:100DE0002F7C2FC081FF94968B9694968B8601EE74
:100DF00057F0D8901E34E926000EEA22EECF04F018
:100E0000EFCF05F004502124006E05502220016E22
:100E1000000E2320026E000E2420036E03C03EF05D
:100E200002C03DF001C03CF000C03BF06FD0020EAC
:100E30002B5C35E11BB40CD02F9A2FC081FF949608
:100E40008B9694968B864268416840683F6826D0AE
:100E50002F7A2FC081FF94968B9694968B8601EE05
:100E600057F0D8901F34E926000EEA22EECF04F0A6
:100E7000EFCF05F004502124006E05502220016EB2
:100E8000000E2320026E000E2420036E03C042F0E9
:100E900002C041F001C040F000C03FF037D0030E67
:100EA0002B5C34E11BB60CD02F982FC081FF949699
:100EB0008B9694968B86466845684468436826D02E
:100EC0002F782FC081FF94968B9694968B8601EE97
:100ED00057F0D8902034E926000EEA22EECF04F035
:100EE000EFCF05F004502124006E05502220016E42
:100EF000000E2320026E000E2420036E03C046F075
:100F000002C045F001C044F000C043F016D824AE42
:100F10000BD0246A236A226A216A1B6A00EE37F02A
:100F2000200EEE68E82EFDD706D024AE04D0246A49
:100F3000236A226A216A11EF01F02B682A8E0B6A5C
:100F4000040E0B5C33E2D8900B34E96EEA6AEA36A1
:100F5000E936EA36370EE926000EEA22EFCF00F036
:100F6000ECCF01F0ECCF02F0ECCF03F02750005CA7
:100F700028500158295002582A50035815E2D89099
:100F80000B34E96EEA6AEA36E936EA36370EE926C4
:100F9000000EEA22EFCF27F0ECCF28F0ECCF29F0BB
:100FA000ECCF2AF00BC02BF00B2ACAE31200200E64
:100FB000115C03E112C01DF011D0210E115C03E1A0
:100FC00012C01EF00BD0220E115C03E112C01FF004
:100FD00005D0230E115C02E112C020F0116812004E
:100FE000156812001768120016681200010E135CD3
:100FF00017E114C02CF01450FF082D6E030ED8A07A
:10100000FF0F2E6E00EE2DF0CF0EBD16EE38300B1A
:10101000BD12ED30F36EEF30BE6EF332BE3234D01F
:10102000420E135C08E1145203E11A902FD802D04B
:101030001A80899A29D07B0E135C26E18A6A9496DD
:101040008B9694968B8692908990929089809292BA
:1010500089929292898292948994929489843A682E
:101060003968386837683E683D683C683B68426864
:10107000416840683F6846684568446843681B6A41
:101080002F6A306A316A326A13681200898A2F6ABD
:10109000306A316A326A8A6A94968B9694968B8605
:1010A000929089909290898092928992929289826C
:1010B00092948994929489841A6A570E2C6E2C50BB
:1010C000FF082D6E030ED8A0FF0F2E6E00EE2DF040
:1010D000CF0EBD16EE38300BBD12ED30F36EEF3093
:1010E000BE6EF332BE323A683968386837683E6897
:1010F0003D683C683B684268416840683F684668B4
:101100004568446843681B6A1D6A1E6A1F6A206A34
:1011100012000101586957695C0E5A6F7A0E596FB7
:10112000590E5C6F850E5B6F580E5E6F140E5D6F0F
:10113000560E606FA90E5F6F550E626F430E616FA2
:10114000530E646FE30E636F520E666F890E656F08
:10115000510E686F350E676F4F0E6A6FE60E696F3E
:101160004E0E6C6F9C0E6B6F4D0E6E6F580E6D6F4A
:101170004C0E706F190E6F6F4A0E726FDF0E716F2B
:10118000490E746FAA0E736F480E766F7A0E756FE4
:10119000470E786F4F0E776F460E7A6F290E796F74
:1011A000450E7C6F080E7B6F430E7E6FEB0E7D6FDE
:1011B000420E806FD30E7F6F410E826FBF0E816F24
:1011C000400E846FB00E836F3F0E866FA50E856F45
:1011D0003E0E886F9E0E876F3D0E8A6F9C0E896F44
:1011E0003C0E8C6F9E0E8B6F3B0E8E6FA40E8D6F20
:1011F0003A0E906FAE0E8F6F390E926FBC0E916FDC
:10120000380E946FCE0E936F370E966FE30E956F78
:10121000360E986FFD0E976F360E9A6F1A0E996FF5
:10122000350E9C6F3B0E9B6F340E9E6F5F0E9D6F55
:10123000330EA06F870E9F6F320EA26FB20EA16F9A
:10124000310EA46FE10EA36F310EA66F140EA56FC1
:10125000300EA86F490EA76F2F0EAA6F820EA96FCE
:101260002E0EAC6FBE0EAB6F2D0EAE6FFD0EAD6FC2
:101270002D0EB06F3F0EAF6F2C0EB26F850EB16F9B
:101280002B0EB46FCD0EB36F2B0EB66F180EB56F5D
:101290002A0EB86F670EB76F290EBA6FB80EB96F06
:1012A000290EBC6F0C0EBB6F280EBE6F620EBD6F99
:1012B000270EC06FBC0EBF6F270EC26F180EC16F16
:1012C000260EC46F760EC36F250EC66FD80EC56F7F
:1012D000250EC86F3C0EC76F240ECA6FA20EC96FD1
:1012E000240ECC6F0B0ECB6F230ECE6F760ECD6F10
:1012F000220ED06FE40ECF6F220ED26F540ED16F3C
:10130000210ED46FC60ED36F210ED66F3B0ED56F54
:10131000200ED86FB20ED76F200EDA6F2B0ED96F5A
:101320001F0EDC6FA60EDB6F1F0EDE6F240EDD6F4F
:101330001E0EE06FA30EDF6F1E0EE26F250EE16F33
:101340001D0EE46FA90EE36F1D0EE66F2E0EE56F06
:101350001C0EE86FB60EE76F1C0EEA6F3F0EE96FCA
:101360001B0EEC6FCB0EEB6F1B0EEE6F580EED6F7E
:101370001A0EF06FE80EEF6F1A0EF26F790EF16F22
:101380001A0EF46F0B0EF36F190EF66FA00EF56FB9
:10139000190EF86F360EF76F180EFA6FCE0EF96F42
:1013A000180EFC6F680EFB6F180EFE6F030EFD6FBC
:1013B000170E0201006FA00E0101FF6F170E020150
:1013C000026F3F0E016F160E046FDF0E036F160ED5
:1013D000066F800E056F160E086F240E076F150E30
:1013E0000A6FC80E096F150E0C6F6E0E0B6F150E7F
:1013F0000E6F160E0D6F140E106FBF0E0F6F140EC2
:10140000126F690E116F140E146F150E136F130EF9
:10141000166FC20E156F130E186F710E176F130E25
:101420001A6F210E196F120E1C6FD20E1B6F120E47
:101430001E6F840E1D6F120E206F380E1F6F110E5F
:10144000226FED0E216F110E246FA30E236F110E6C
:10145000266F5A0E256F110E286F120E276F100E71
:101460002A6FCC0E296F100E2C6F870E2B6F100E6B
:101470002E6F420E2D6F0F0E306F2F69326FBD0E23
:10148000316F0F0E346F7C0E336F0F0E366F3D0EC3
:10149000356F0E0E386FFE0E376F0E0E3A6FC00EA0
:1014A000396F0E0E3C6F830E3B6F0E0E3E6F470E74
:1014B0003D6F0E0E406F0C0E3F6F0D0E426FD20E41
:1014C000416F0D0E446F990E436F0D0E466F610E06
:1014D000456F0D0E486F2A0E476F0C0E4A6FF40EC3
:1014E000496F0C0E4C6FBE0E4B6F0C0E4E6F8A0E7A
:1014F0004D6F0C0E506F560E4F6F0C0E526F230E29
:10150000516F0B0E546FF10E536F0B0E566FC00ED2
:08151000556F00011200FFD726
:020000040030CA
:0300010006160ED2
:020005008580F4
:060008000FC00FE00F40E5
:00000001FF
